:030000000219FDE5
:03000B000200AA46
:03002B0002015F70
:03005B000202E7B7
:030073000202CDB9
:1000800002030406080C10182030406080040608A3
:100090000C10182030406080A0C000070F1F3F0DDB
:1000A0000D04050D050205030302C2AFC0D0C0E078
:1000B000206217E5256002E473E525F4F58A758B67
:1000C00000D262D0E0D0D0D2AF3285268AC262E5BB
:1000D00026F4602F758B00D0E0D0D0C292C291C2BE
:1000E00090D2AF32C292C291C290206E0C206609AB
:1000F0007405D5E0FDE57E4290758B00D0E0D0D050
:10010000D2AF32758A00C28DD26201F901B930686E
:1001100005206602D29201B9306805206602D291AC
:1001200001B9306805206602D29001B9C2953068E5
:100130000A2066077446D5E0FDD29201B9C2943018
:10014000680A2066077446D5E0FDD29101B9C293D2
:1001500030680A2066077446D5E0FDD29001B9C226
:10016000AFC2AD53E6EFC0D0C0E0D2D3D2AFC2CE63
:10017000E52A6007207449152A21C07800790020FB
:10018000742EE580307E01F430E70278FF53DACF39
:10019000207E0343DA20307E0343DA10C2D8C271D6
:1001A000E580307E01F430E70279FFC3E89970CB37
:1001B000306103752A18207403752A18885FD2707D
:1001C00020740DE52B6004152B21D043DA01C2D831
:1001D000207002412EA85F206102C270207436791F
:1001E00082B70431C3E894F0400374F0F8E8C454D3
:1001F0000F28F87984B703024115C313C31387216D
:10020000200802C313200A06C3C898F8411528F82D
:10021000500374FFF88822E52D54066011E533C3BE
:1002200013C31324062522F52250037522FF78827A
:10023000B6044E852224A824C3E52495644002A870
:1002400064C3E895664002A8668825E569700241A6
:100250007FC3E8AA699A5003E8FAE4F9EAC333FBDA
:10026000E56BF45B29400D256AF8E56A6002156AC2
:10027000400B417F0AC3E56A9A5002056A78FF88FD
:1002800026C3E52594404002D26420CF0AD0E0D0B6
:10029000D043E610D2AD32C2CF053A7801E52A60EC
:1002A00005307402152AC3E55F94014005756200AC
:1002B00041C3756300756C00E5622401F56250036B
:1002C0007562FFD0E0D0D043E610D2AD32C2AFC0ED
:1002D000D053E67FC2607591008556948557957519
:1002E0009104D0D0D2AF32C2AF53E6EFC2ADC0D08E
:1002F000C0E0C0F0D2D3D2AFA8FBA9FCC2D8307105
:1003000002614E53DACF207E0343DA10307E03437E
:10031000DA20D271E580307E01F420E70261258881
:10032000278928A17553DACF207E0343DA20307E57
:100330000343DA10C2D8C271307402A1617800E5BB
:1003400080307E01F430E702A161885FA14953DA71
:10035000CF207E0343DA20307E0343DA10C27120BF
:100360006102812753DACF207E0343DA10307E0307
:1003700043DA20C2D8D271885A895BC3E89558F80D
:10038000E99559F97B007E087A00C3E8948CE994DA
:10039000005005755E008119882178A2E6A82160C9
:1003A00055C3E894C8E994005008E4D2E4FB7A0A03
:1003B00061F4C3E89468E994015008E4D2E3FB7A5D
:1003C0000F61F4C3E894D0E994025008E4D2E2FB50
:1003D0007A1E61F4C3E894A0E994055008E4D2E1E0
:1003E000FB7A3C61F4C3E89498E994085008E4D29D
:1003F000E0FB7A787E00C3E8955CFCE9955DFD3012
:10040000E70AECF42401FCEDF43400FD755E00C352
:10041000EC9AED9E5003755E01885C895D855A58A3
:10042000855B597802A149C3E89527F8E99528F931
:10043000307C02A12D307B02A12D307A02A1262032
:100440007502814AE9FDE8FC8169E9C313F9E81303
:10045000F8307902A126E9C313F9E813F8307802DD
:10046000A126E9C313FDE813FC206126C3EC941C0C
:0E047000ED940240028180ED7018C3EC94C838
:10047E0050120529C3E529940A5002A161755F0047
:10048E00D270A161E529600215297888E6F9740019
:10049E00207F087896B90302789EE624FAFEE434AB
:1004AE0000FFC3EC9EFCED9FFD9208B90310A2085D
:1004BE005007207609D27681CC307602C276A20819
:1004CE005016B9030DECF42401FCEDF43400FD02DA
:1004DE0004E678007900A12DB90315EC33FCED3359
:1004EE00FDC3EC940AFCED9400FD50047C007D00ED
:1004FE00C3EC94FFED9400400678FF7900A12DEC3B
:10050E008575F0A4C5F0A2F733F879004003020513
:10051E004978FF7900020549E9C313F9E813F83069
:10052E007C0EE9600278FFC3E81338F8E43400F972
:10053E00C3E894FFE99400400278FF885FD27020F0
:10054E006102A161741FF4552F4BF52FC274EB702D
:10055E0002D274752A18307403752A0A306102A10A
:10056E007520740353DAFE207403752B06D0F0D079
:10057E00E0D0D0D2AD43E6103279010205A5790361
:10058E000205A5790A0205A5791E0205A579640260
:10059E0005A579C80205A57817E4D5E0FDD8FAD9E6
:1005AE00F6227A147B780205CC7A107B8C0205CC6D
:1005BE007A0D7BB40205CC7A0B7BC80205CC79028E
:1005CE00B27DE4C294D5E0FDD291D5E0FDC291D5C5
:1005DE00E0FDD294D5E0FDD292E576D5E0FDC29253
:1005EE007496D5E0FDD9D9EAF8D5E0FDD8FBDBCE7F
:1005FE00C29422C37C007D0075F00005F0EA33FA48
:10060E00EB33FB50F6EB13FBEA13FAC3E9FFE8FEFC
:10061E00E89AF8E99BF95004EFF9EEF8B3EC33FCE5
:10062E00ED33FDD5F0DFEDF9ECF822E889F08A2004
:10063E00D2D4F8A9F07B0030F70B7BFFF42401F83D
:10064E00E9F43400F9E88520F0A4ADF0F8E985204E
:10065E00F0A4AFF0FEED2EF974003FFA7C04C3EA6D
:10066E0013FAE913F9E813F8DCF48BF030F70AE823
:10067E00F42401F8E9F43400F9E889F0C2D4F8A9B9
:10068E00F0227882B604030206EBC3E55F940140C4
:10069E00030206B5852224E4F545F546F547F548EF
:1006AE00F549C26D0206EB7882E6FCD26DE522F5C5
:1006BE0023783879C7AA40AB41C3EB13FBEA13FA90
:1006CE00EC146013C3EB13FBEA13FAEC141460077B
:1006DE00C3EB13FBEA13FAD1018845894622C3E521
:1006EE00459523F8E5469400F9500CC3E89480E94B
:1006FE0094FF401602071CC3E8947FE99400500350
:10070E0002071C787F790002071C788079FF884ADF
:10071E00894B22E54A2547F8E54B3548F9854B20AC
:10072E00E4300701F43549FA30E709C3EA94F040A2
:10073E001502075AC3EA940F500302075A78FF793D
:10074E00FF7A0F02075A780079007AF0C3E52495F4
:10075E0064500AC374019524500B020778E54B20B0
:10076E00E70E020778E54B30E706884789488A4945
:10077E002278A4E6FAC3E54A33F8E54B33F9D139CA
:10078E00E930E70BC3E89480E994FF4013E1B2C36C
:10079E00E8947FE994005002E1B2787F7900E1B2EB
:1007AE00788079FFE820E715C3E52398F84009C360
:1007BE00E8940140030207D978010207D9E8F4242E
:1007CE00012523F840030207D978FF884C2278A52B
:1007DE00E6FAA848A949D139E930E70CC3E89401F3
:1007EE00E994FF401602080DC3E894FFE994005007
:1007FE000302080D78FF790002080D780179FFE9F0
:10080E0020E715C3E54C98F84009C3E8940140036E
:10081E000208347801020834E8F42401254CF8402B
:10082E000302083478FF88242278FFC26420693DD1
:10083E00206A12D264C3E541940A4009C3E52594A7
:10084E00405002C26479A1E76023E541601F74FF46
:10085E008541F0848539F0306A0375F005A4F8C53A
:0F086E00F0600278FFC3E895675002A8678866BC
:10087D0022C3E5409440E5419401E566500314011F
:10088D008F046002F566220208972275E89022789F
:10089D0083E6FFE5E820ECF7A8BDA9BE0573C3E527
:1008AD007394084052757300E9FA79A0E76044EA41
:1008BD007007E574601B0208D2C3E895746010E5FB
:1008CD00745006600C140208DE0460F90208DEE5BF
:1008DD0074F574C3946D401B7564C0C394044013C8
:1008ED00756480C39404400B756440C39404400345
:1008FD0075640075BB0622E5642410500274FFF583
:10090D00647982B70402212BC3A864E524985002B0
:10091D00A824C3E895664002A86688258826E57355
:10092D00B4070375BB1022743279A687F0A4C5F005
:10093D00A2F733F8C3E895644002A864882288249E
:10094D00882588268867227540007541F022C2AF40
:10095D0075C820A8CCA9CDAA3A30CF010A75C824F4
:10096D00D2AFAB3BAC3C883B893CC3E89BF8E99CE0
:10097D00206908F9306702417021CDAD3D8A3DF9FE
:10098D00EA9DFA600478FF79FFAE3EAF3F8B3E8C57
:10099D003FC3EC9FFCC3E99CF542A83BA93CC3E8CF
:1009AD009EF8E99FF9C3E54113FBE54013FAE82AE8
:1009BD00F540E93BF54150067540FF7541FF411784
:1009CD00AA40AB41AC40AD417E047F02C3EB940421
:1009DD0040021E1FC3EB940840021E1FC3ED13FD02
:1009ED00EC13FCDEF7C3EA9CFAEB9DFBEF6009C349
:1009FD00E913F9E813F8DFF7EA28FAEB39FB8A4037
:100A0D008B4150067BFF8B408B41C3EB9402500210
:100A1D00D2673069047F0341427892E6FFC3E53720
:100A2D00948240110FC3E53794A040010FC3EF949A
:100A3D000640027F057E07E541C4540FF9E541C428
:100A4D0054F0F8E540C4540F28F8C3E89EFAE99431
:100A5D0000FB4009C3EA9402EB940050047A02E4CF
:100A6D00FB41BCAA40AB41EBC4FEEAC4540F4EFCA3
:100A7D00C3EA9CFAEB9400FBC3E813C313F8EA280E
:100A8D00FAEB3400FB8A408B41C3EB94024002C267
:100A9D00677807EBC4FE7B00EAC4540F4EFAC3EA35
:100AAD0098FA4005C3940250027A027892E6FF301C
:100ABD00600241BC855256855357D26043E680C3D0
:100ACD00E49AF8E49BF93067026156E8FAE9FBD342
:100ADD00E913FDE813FC88528953C3EF9403603882
:100AED00EF20E00DE82CF8E93DF9ECFAEDFB020BF7
:100AFD0011E828F8E939F9C3E82402F8E93400F9D6
:100B0D007AFE7BFFC3EF9403400E8A548B55884EBB
:100B1D00894F8C508D51618A885489558A4E8B4FDF
:100B2D008C508D51306920C3E53394034019E54253
:100B3D00A2E713F8E555F4240138400B20E70875BA
:100B4D0054FFF42401F555618AE8FAD3E813FC88C3
:100B5D0052C3EF94036020EF20E007E82CF8ECFA85
:100B6D006176E8282402F87AFEC3EF940340088AE0
:100B7D0054884E8C50618A88548A4E8C50E56BC3D4
:100B8D00335002646BF56B3060026194753402D2A0
:100B9D006043E680E52D54066026A840A941C3E9CF
:100BAD0013F9E813F8C2AF53E67F759100C3E498CB
:100BBD00F594E499F595759104D26043E680D2AF32
:100BCD0022D265754400752000306B0375204002FC
:100BDD000BEDD265754400752040306B0375200018
:100BED00D2AF7801206722E52D54066002C265C39D
:100BFD00E541940540137802940540087803940567
:100C0D0040027806306902780A206019E5446015C3
:100C1D0030690AC3E53394034003D53406D2AFD20D
:100C2D006C81BF719CD2AF0000C2AF206726E54139
:100C3D00C3FB940F40027B0FEB240530730123306F
:100C4D006A02742820620123F93069027982E58BEA
:100C5D00C39940B50544E59BF45440B5200281A9E4
:0D0C6D0030690A08C3E8940A4001088116A6
:100C7A0020650261EDC26553E67F75910030671009
:100C8A007594007595FE759104D26043E68061ED16
:100C9A00AE40AF41C3E49EF594E49FF5958190C3BD
:100CAA00E5339402500261ED30650261EDD80281AC
:100CBA00BD8116C26C53E67F7591008554948555A3
:100CCA0095759104854E56854F57D26043E680D27A
:100CDA00AFE52D54066008206A020533020CF9308C
:100CEA006C0D206B0A2065071581158102155F229C
:100CFA0078003064053065027801E53775F007A49D
:100D0A00F9E5F028F5F0E9A2F013A2F113A2F21323
:100D1A00F537C394785003753778C3E5379538406B
:100D2A0008D266C292C291C290306002A133855045
:100D3A0056855157D26043E68022207D11C2AF7595
:100D4A004302C294D295D2AF759F11020F13C2AF5C
:100D5A00754302C294D293D2AF759F11020F13301A
:100D6A007243207D20C2AF75430390013D757E100A
:100D7A00C290C293306204D291A187D294D2AF7545
:100D8A009F01020F13C2AF75430390013D757E1098
:100D9A00C292C295306204D291A1A7D294D2AF7501
:100DAA009F21020F13207D17C2AF754303900118CC
:100DBA00C290306202D291D2AF759F01020F13C264
:100DCA00AF754303900118C292306202D291D2AF3A
:100DDA00759F21020F13207D11C2AF754304C2957E
:100DEA00D293D2AF759F21020F13C2AF754304C2CB
:100DFA0093D295D2AF759F01020F13307243207DB3
:100E0A0020C2AF75430590012C757E20C291C29411
:100E1A00306204D292C123D295D2AF759F11020FCC
:100E2A0013C2AF75430590014E757E08C291C294F4
:100E3A00306204D290C143D293D2AF759F11020F90
:100E4A0013207D17C2AF75430590010EC29130621F
:100E5A0002D292D2AF759F11020F13C2AF7543052A
:100E6A00900122C2913062EBD290D2AF759F1102EB
:100E7A000F13207D11C2AF754306C293D294D2AF2D
:100E8A00759F01020F13C2AF754306C295D294D261
:100E9A00AF759F21020F13307242207D20C2AF75B9
:100EAA00430190014E757E08C292C295306204D207
:100EBA0090C1BFD293D2AF759F21020F13C2AF75F3
:100ECA00430190012C757E20C290C293306204D2F5
:100EDA0092C1DFD295D2AF759F01E113207D16C270
:100EEA00AF754301900122C292306202D290D2AF12
:100EFA00759F21E113C2AF75430190010EC2903074
:100F0A006202D292D2AF759F01C2662290010C751D
:100F1A007E00C292C291C290C295C294C293C2622A
:100F2A0022788076090876090876040876FF08761A
:100F3A00030876FF08760B08760108760108760121
:100F4A00788C76010876FF0876FF0876FF0876FF28
:100F5A000876FF0876030876FF0876FF0876FF080A
:100F6A0076250876D008762808765008760408761A
:100F7A00FF08760208760008767A0876FF08760176
:100F8A00087601087600087603227887E6FFC2729F
:100F9A007888E6C394036008C27DE630E102D27D18
:100FAA00C27E7889E630E102D27EC3EF94026008FD
:100FBA00758E01D273020FC7758E00C273227880B4
:100FCA00E6149000809378A4F67881E61490008065
:100FDA009378A5F67886E61490008D9378A6F6782D
:100FEA009CE67538FF75390CB402067538A0753958
:100FFA000AB4030675388275390578A3E614900099
:10100A009A93F569120F1622227896E6FA7897E6ED
:10101A00FB7888E6B40305C3EB940EFB307F047AB1
:10102A00007BFFC3EB9AFCC3948250027C827575E5
:10103A00000575EC8575F0A4C3E5F0947D40F222B5
:10104A00D27F11131205967A007B007C1012058C50
:10105A00E55F2AFA74003BFBDCF37C04C3EB13FB69
:0D106A00EA13FADCF7FEC27F111322E5EF56
:1010770020E6037520000520903FFFE52014600659
:10108700901DFF1460009304600375EF1053D9BFE0
:101097007581C043FF8012058775EF0043B203E5F2
:1010A700B3240420E70DF521E5E320E0068521B30D
:1010B70043E301120F167580FF75A40075F1907553
:1010C700D47F75900075A53F75F23F75D50075A65D
:1010D7000175E241E4F8F6D8FD756B01120F2B128A
:1010E70015A178988676753001C2AF1205A0120552
:1010F700B01205961205B71205961205BE1205968F
:10110700C2AF78FA79FA308707D9FBD8F7021C0003
:10111700120F94120FC81112111378988676120FB6
:101127001675885075891275C82475910475D8404D
:1011370075A82275B80275E690759B80759D007538
:10114700D10E75BC5875BB0675BA1175E8801205C6
:1011570087D2AF12089453DACF207E0343DA2030C8
:101167007E0343DA1043DA01C2D8C2711205A0D256
:10117700617B037A0CE55E70077A0CDB03021107CB
:10118700120596207003021107C270E55FC394022F
:1011970040E1E52F541F856160F561B560D5DAD56B
:1011A700C26153DACF207E0343DA20307E0343DA6D
:1011B70010C2D8C27178A2E67008D274E52F54E045
:1011C700F52FC27575290012059B307409C3E529EF
:1011D700940A4002D27512058C78023074027800A6
:1011E700C3E55F9840F0C2AF1205B01205B0120513
:1011F700B0D2AF1205A0754D007888E6B40302415E
:10120700DE12058C788CE6C3940150030212DEE5EA
:1012170030C3940150030212DE207435C3E55F9496
:10122700FF50030212DEC2AF1205C5D2AF12059BF3
:10123700C3E55F940150EFC2AF1205B012059112DA
:1012470005B0D2AF12059BC3E55F94FF40E90217D3
:10125700497F02D27F111312059BC2AFC27F1113C0
:10126700AE5FC3E55F947FD2AF4076120587C2AF0A
:101277001205C5D2AFDFDC114AC3EE94057897F6A5
:101287001205A01215E31216CC7F0AD27F11131292
:10129700059BC2AFC27F1113AE5FC3E55F947FD2D8
:1012A700AF50E6120587C2AF1205B01205911205BD
:1012B700B0D2AFDFD6114AEE24057896F61205A014
:1012C7001215E31216FB12059B1113C3E55F94FF7A
:1012D70050024120021749C3E55F954D4003855FE2
:1012E7004D12059B78017988E7B403027805C3E5B9
:1012F7005F9840024100C2AF1205C51205C512052D
:10130700C5D2AF1205A0753000E4F531F5320531CD
:10131700E531F470390532789AE678191460127855
:101327003214600D787D14600878FA146003753202
:1013370000C3E53298401715327531B4789986762F
:10134700C2AF1205C5D2AF7898867612059B1205F3
:1013570091E52A700530740221077801207402781C
:1013670006C3E55F9840A77888E6C3940360031235
:10137700059BE52A7003021107C2AF120F16E4F5A9
:1013870022F523F524F525F526F56AD2AF7885E60B
:10139700C333F568E4F545F546F547F548F549F5EE
:1013A70073F52CF52DF53775730875BB1012058786
:1013B700120898E5E820ECFBA8BDA9BEE97001F882
:1013C700887412089C75730875BB107887E6FE76DB
:1013D70002120F947887EEF6C2AF7564FF120934D4
:1013E700852264852265852266D2AF752201752420
:1013F7000175250175260185636C756D017888E691
:10140700B40307C27D307602D27DD268D2697533C4
:1014170000120E7C120EA112095412095B12095414
:1014270012095B12095402143DC2AF120F94D2AFD6
:1014370075730075BB06120BDF120690120CFA12B9
:101447000D4412095B120BCE306D031206EC2067B8
:101457000312083730670312087E120CFA120D695F
:0F14670012095B120BDF306D03120721120CFA12
:10147600120DE012095B120BCE306D0312077F12BC
:101486000CFA120E0512095B120BDF306D03120700
:10149600DC120CFA120E7C12095B120898120BCEA3
:1014A600120CFA120EA112089C12095B3069352043
:1014B6006B3285676485676585636C756D01791820
:1014C6007A0CC3E53399400FC269D26A8A358567BB
:1014D600648567660214EAC3E55F9401400302145B
:1014E6003D021567306A1B206B18E535147004C27F
:1014F6006A8130F535C3E55F9401400302143D026D
:101506001567753600C3E56278FA9850543074044E
:10151600E52A604D7888E6B40317207D0520760716
:10152600A137307602A137206B07D26B85676481BD
:101536007C78F0306B058567647820C3E541985068
:1015460002813D306B1BC26BC27D307602D27DD2EA
:101556006A753512856764813D0536E55F6002A1CF
:101566006A753600C2AF120F167887E6FE7602124B
:101576000F947887EEF6E4F522F523F524F525F5A4
:1015860026F568C268D2AF120587120F16307409A5
:10159600C3E5369405400221076110901A0D7820A4
:1015A600121625E520B4550CA3121625E520B4AA7B
:1015B600030215C3120F2B1215E30215E2901A034C
:1015C60078807B0A121625A308DBF9901A0F788C0F
:1015D6007B18121625A308DBF9901A2722C2AF1230
:1015E600166412163E901A00740E12162AA374047C
:1015F60012162AA3741412162A901A0378807B0AEC
:10160600121629A308DBF9901A0F788C7B1812168C
:1016160029A308DBF9121677121655901A2722E429
:1016260093F622E6438F01538FFD75EF0275B7A53A
:1016360075B7F1F0538FFE22438F02438F0175EF8A
:101646000275B7A575B7F1901A0DF0538FFC22906D
:101656001A0D7455D12A901A0E74AAD12A227A30FC
:1016660079D07820901A40D125E520F709A3DAF73A
:10167600227A3079D0901A40E7D12A09A3DAF922E2
:10168600AB77A878BB01027980BB02027981BB03E4
:10169600027982BB04027984BB05027986BB060205
:1016A6007992BB07027987BB080279A3BB09027945
:1016B6009CBB0A027988BB0B027989E8F7227C0574
:1016C6001205A0DCFB22C2AF1205B01205B7120547
:1016D600BE1205C51205911205B01205B71205BE58
:1016E6001205C51205911205B01205B71205BE12F4
:1016F60005C5D2AF22C2AF1205C51205BE1205B787
:101706001205B01205911205C51205BE1205B712D3
:1017160005B01205911205C51205BE1205B71205D0
:10172600B0D2AF22AE77AF78C2AF1205B01205B015
:101736001205B0120591DEF21205C5120591DFF809
:10174600D2AF22D1CCD1C4D1C475770175780175D9
:101756007900F12A7C05AD5F1205A0C3ED955F7097
:10176600F5C3E55F9401400AC3E55F94FF4032028A
:101776001785D186B1E3D1CCC2AF75EF10D1C4DCE9
:10178600D50579C3E5799403500280C6D1C405789E
:10179600E5771490009F93F808C3E5789850028087
:1017A600AED1C4D1C40577C3E577940C5002809CB2
:0C17B600120F2BB1E3C2AF75EF10D1C4CD
:0319FD0002107560
:101A00000E0414090904FF03FF0B01010155AA018B
:101A1000FFFFFFFFFF03FFFFFF25D0285004FF0259
:081A2000007AFF01010003FF41
:101A400023585031324123202020202020202020E4
:101A500023424C48454C4923463333302320202031
:101A60002020202020202020202020202020202076
:101C0000C2AFC2D353D9BF7581C043B20343FF8073
:101C1000752438752503B1C975EF0275E24043F1AB
:101C20008053A47F75D400D2877DFA780379E67C4F
:101C300010752200752300901DD67B0675249875BB
:101C400025013087028142208708D8FBD9F9DCF7CB
:101C500081B4308708D8FBD9F9DCF781B4B189E4C5
:101C600093A3C39A6004DDC381B4DBDBB17B600264
:101C7000812B7B08E493FAA3B15CDBF87A30B15C8A
:101C8000752200752300B17BEAFCEBFDC3ED94FEE9
:101C9000400EB17B8A278B28ED30E0048A828B834B
:101CA000B17B7AC270D8C3ED94FE601350CEBD00F4
:101CB00025EC60097520007521FF0200008100A855
:101CC00027A9280809D804D90281D3B17FEA89AAB3
:101CD000F281C50D81A0C3ED94035049EDA2E092BD
:101CE000007AC5C3E5829400E583941C50902000DF
:101CF00010438F02438F0175B7A575B7F1F030001F
:101D00001FA827A9280809438F01538FFDD804D99C
:101D100002A12089AAE275B7A575B7F1F0A3A10DBC
:101D2000538FFC817C7AC1BD030CE493A3FAB140CC
:101D3000DCF8B138817C817EAA22AB23B15CEBFA5E
:101D4000EA6222752608C3E52313F523E52213F57D
:101D50002250066323A0632201D526EAB1C9B1C986
:101D600075260AEAF4200102D287300102C287B147
:101D7000C9C3134002C201D526EB22B17FEAFB2082
:101D80008702A17F308702A184752608AE24AF2583
:101D9000C3EF13FFEE13FEB1CDB1C9C3EA13308711
:101DA000024480FA30E703632201C3E52313F523DD
:101DB000E52213F52250066323A0632201D526D91C
:101DC000E52265236523F52222AE24AF250E0FDE22
:101DD000FEDFFCD20122424C48656C693437316326
:041DE000F3300601D5
:00000001FF
